:0200000480007A
:100000006F008004732F2034930F80006308FF0378
:10001000930F90006304FF03930FB0006300FF038E
:10002000130F000063040F0067000F00732F2034CC
:1000300063540F006F00400093E19153171F0000BD
:1000400023223FFC6FF09FFF93000000130100008C
:10005000930100001302000093020000130300004C
:100060009303000013040000930400001305000034
:10007000930500001306000093060000130700001C
:100080009307000013080000930800001309000004
:1000900093090000130A0000930A0000130B0000EC
:1000A000930B0000130C0000930C0000130D0000D4
:1000B000930D0000130E0000930E0000130F0000BC
:1000C000930F0000732540F16310050097020000B4
:1000D000938202017390523073500018970200000F
:1000E00093824202739052309B021000939252030B
:1000F0009382F2FF7390023B9302F0017390023AF5
:100100007350403097020000938242017390523046
:10011000735020307350303093010000970200007C
:10012000938282EE73905230130510001315F5017F
:10013000635C05000F00F00F930110009308D005D9
:10014000130500007300000093020000638A0200A0
:1001500073905210B7B200009B82921073902230BD
:100160007350003097020000938242017390123462
:10017000732540F173002030B710FF009B8000F022
:1001800013C7F0F0B7F300FF9B83F3009301200047
:100190006316771CB710F00F9B8000FF13C7000F8A
:1001A000B713F00F9B8303F0930130006318771AA5
:1001B000B710FF009B80F08F13C7F070B713FF00DC
:1001C0009B8303FF93014000631A7718B7F00FF089
:1001D0009B80F00013C7000FB7F30FF09B83F30F62
:1001E00093015000631C7716B7F000FF9B800070EE
:1001F00093C0F070B7F300FF9B83F300930160009E
:10020000639E701413020000B710F00F9B8000FF74
:1002100013C7000F130307001302120093022000FC
:10022000E31452FEB713F00F9B8303F093017000A9
:100230006316731213020000B710FF009B80F08F4B
:1002400013C7F0701300000013030700130212001D
:1002500093022000E31252FEB713FF009B8303FFBB
:1002600093018000631C730E13020000B7F00FF0BF
:100270009B80F00013C7000F130000001300000064
:10028000130307001302120093022000E31052FE32
:10029000B7F30FF09B83F30F930190006310730C7F
:1002A00013020000B710F00F9B8000FF13C7000F70
:1002B0001302120093022000E31652FEB713F00F50
:1002C0009B8303F09301A000631A770813020000D8
:1002D000B710FF009B80F0FF1300000013C7F00071
:1002E0001302120093022000E31452FEB713FF0022
:1002F0009B8303FF9301B000631277061302000093
:10030000B7F00FF09B80F000130000001300000016
:1003100013C7000F1302120093022000E31252FED3
:10032000B7F30FF09B83F30F9301C00063187702BC
:100330009340000F9303000F9301D000639070026D
:10034000B700FF009B80F00F13C0F0709303000014
:100350009301E00063147000631030020F00F00F8F
:10036000638001009391110093E111009308D0057F
:1003700013850100730000000F00F00F93011000BF
:100380009308D0051305000073000000731000C02F
:10039000000000000000000000000000000000005D
:1003A000000000000000000000000000000000004D
:0C03B00000000000000000000000000041
:1010000000000000000000000000000000000000E0
:1010100000000000000000000000000000000000D0
:1010200000000000000000000000000000000000C0
:1010300000000000000000000000000000000000B0
:081040000000000000000000A8
:040000058000000077
:00000001FF
